:020000020000FC
:1000000040C018951895D8C2189518951895189548
:100010001895189518951895189518951895010222
:1000200004080000808080800000010101010000C0
:10003000000000000000007F40007F40007F400083
:100040007F40000306090C101316191C1F222528D7
:100050002B2E313336393C3F414447494C4E5153A6
:1000600055585A5C5E60626466686A6B6D6F707149
:100070007374757678797A7A7B7C7D7D7E7E7E7FDF
:100080007F7FAA240FE50DBF02E00EBF00E806BD8A
:1000900000E006BD379843E0A0E6BB27EEE1F0E0C4
:1000A00002C005910D93E238E1F738D202E026D282
:1000B0006CD1BED1E4EAF1E02ED1E6E9F1E02BD13A
:1000C000E4EAF1E028D1E6E9F1E025D15ED103E0F0
:1000D000B02E25D103E0B02E22D190E107E6B02E5C
:1000E00024D10FEDE7D19A95C9F7E6E9F1E013D1F4
:1000F000E4EAF1E010D1E6E9F1E00DD1E4EAF1E063
:100100000AD1ACEBB7E0EFD0EED0EDD0ECD0A0D080
:10011000B9D0A8E7BFE0E7D0B695A795E4D0A7EFA0
:10012000B0E0E1D0ACEBB7E0DED0A7EFB0E0DBD0E1
:10013000B7E0ACEBCBD101D108D16FD06ED0BCD041
:100140000CE0B02EECD003E0B02EE9D00CE0B02EE5
:10015000E6D003E0B02EE3D00CE0B02EE0D008E013
:10016000B02EDDD0B1E0AFEEB1D10FD190E203E31C
:10017000B02EDBD005E99ED19A95C9F734D033D0A3
:1001800032D031D0F2D0F1D0F0D0EFD0F6D0F5D0DF
:10019000F4D0F3D08BCF0412004774D5479A4000B7
:1001A0008540007604120047742B479A4000854032
:1001B0000076004774D5479A405585405576002B08
:1001C00074802B70401785281776020C002B89004D
:1001D0002B85405585A85576020C002B89002B8570
:1001E000C05585285576021900477400479A40008B
:1001F00085A800760219003989003985401C85A838
:1002000055760219003989003985405585A81C7634
:1002100099E0EAE1F2E097D1089501EF80808080D3
:1002200001EF718E808001EF639C808001EF55AA01
:10023000808001EF47B8808001EF39C6808001EFF0
:100240002AD4808001EF1CE380800F781CE380803B
:1002500097E0EAE5F2E077D1089501EF80808080B1
:1002600001EF47638080007C71638080007C2A639B
:100270008080007C71638080007C2A63808001EF35
:100280007163808097E0EEE8F2E05DD1089501EFC0
:100290008080808001EF9CB88080007C9C8E808074
:1002A000007C9CD48080007C9C718080007C9CD4ED
:1002B000808001EF9C8E808096E0E2ECF2E043D1FA
:1002C000089500F88080808000F8AAC6808000F839
:1002D000C6C6808000F8C6C6808000F8AAC68080A6
:1002E00000F880808080AF93BF9395E0E8EFF2E064
:1002F0002AD1BF91AF910895001D55638080001DE4
:100300009CAA8080001D55638080001D9CAA80806F
:10031000001D9CAA80804590B590BCD10895E2EB69
:10032000F1E044244394B6D108959F93EEEBF1E0BD
:1003300044244394AFD19F9108959F93EAECF1E058
:100340004590B590A7D19F9108959F93E8EDF1E076
:100350004590B5909FD19F9108959F93E6EEF1E06F
:100360004590B59097D19F9108959F93E4EFF1E068
:100370004590B5908FD19F9108959F93E2E0F2E070
:100380004590B59087D19F91089583E08F9383E046
:100390008F9399E0ECEDF3E0D6D0AFEEB1E096D0DC
:1003A0008F918A95A9F793E0E2E1F4E0CCD08F91A8
:1003B0008A9561F782E08F9399E0ECEDF3E0C3D08A
:1003C000AFEEB1E083D08F918A95A9F702E1B02E0C
:1003D000A6DF92E0E4E2F4E0B6D008950001808068
:1003E0008080000F39808080000F80808080000135
:1003F00080808080000880C68080000880808080A7
:100400000001808080800008398080800008808022
:100410008080001955AA8080001980808080007C2F
:1004200080808080003E39C6808000F88080808097
:1004300087E08F9383E08F9395E0E2E7F4E083D049
:100440008F918A95C1F783E08F9395E0E0E9F4E01E
:100450007AD08F918A95C1F78F918A9551F783E071
:100460008F9395E0E0E9F4E06ED08F918A95C1F723
:10047000089500098080718E000980808E710009C6
:100480008080718E000980808E71001980808E714D
:10049000000939C6718E000939C68E710009808045
:1004A000718E000980808E71001980808E71119785
:1004B000F1F708950F93BF93AF93B3E1A8E8F7DF87
:1004C0000A95D9F7AF91BF910F910895BF93AF935C
:1004D000B3E1A8E8ECDFAF91BF911197B9F70895A8
:1004E0000F93AF93BF930F930AE0E4DFE9F70F9107
:1004F0000A95C9F7BF91AF910F9108950F93CF93CC
:10050000DF93CAE00F9304E6D5DFCA95E1F70F91B8
:100510000A95B9F7DF91CF910F910895F89434E0DF
:10052000222427B3E0E6FF278191282B3A95E1F7B3
:1005300027BBA0BE28E020BF20E429BFAFBC2FEF1F
:100540002EBD78940895FF93EF939F9309D09F91C8
:10055000EF91FF9106E0E00FFA1D9A95A1F708953B
:1005600034E0C6E60591802E0591702EE894059141
:100570008881081B08F01AF4689400950395069585
:100580000695069516F400950395C45F0883CC5034
:10059000C3953A9559F798E034E0C6E6E2E7FF27BD
:1005A00008818191080F09933A95D1F7B82DA72DAD
:1005B0008DDF9A9589F708950F930FB70F932F93B7
:1005C0008F93EF93FF934423F1F0413009F42BC054
:1005D000423009F441C0433009F042C02394022D57
:1005E000043009F42224ECE6E20D0081002331F00E
:1005F00028B3E0E6E20D0081022B08BBAFBC8EE31E
:100600008EBD44272DC0E6E6E20D808186958EBD25
:1006100041E0AFBC8EB58A1103C08FEF8FBD20C003
:1006200080E488BF1DC0ECE6E20D2081222339F072
:1006300028B3E0E6E20D00810095022308BBE6E660
:10064000E20D00818FEB0E3B10F043E001C042E071
:10065000801B8EBDAFBC04C043E0AFBC0FEF0EBD2E
:10066000FF91EF918F912F910F910FBF0F911895DF
:10067000EF9307FB06FF07C0902E0F7311F4092DAF
:100680000395009503950F73E4E8E00F008107F9E7
:10069000EF910895A8E7B0E09CE005910D939A953D
:1006A000E1F7FF27BB27DD24E8E7A6E694E0392E33
:1006B000C1900D2D0C0DDCDF819107FB0F77992484
:1006C00098E0869508F4900E97949A95D1F7092DA5
:1006D00016F4009503958191080F0D933A9441F714
:0E06E0000EE1E8DEDB0C00F74A94E9F608951F
:00000001FF
